:020000040800F2
:1000000000800020310D0008370D0008730D000836
:1000100000000000000000000000000000000000E0
:10002000000000000000000000000000ED0C0008CF
:100030000000000000000000EF0C0008C90C0008E0
:10004000F10C0008F30C0008F50C0008F70C000890
:10005000F90C0008FB0C0008FD0C0008FF0C000860
:10006000010D0008030D0008050D0008070D00082C
:10007000090D00080B0D00080D0D00080F0D0008FC
:10008000110D0008130D0008150D0008170D0008CC
:10009000190D00081B0D00081D0D00081F0D00089C
:1000A000210D0008230D0008250D0008270D00086C
:1000B000290D00082B0D00082D0D00082F0D00083C
:1000C0004543532E46573A30312E30302E303100D2
:1000D0000120C006014908607047C04608ED00E0F5
:1000E00010B51D4CA0688006400F411E032923D87F
:1000F0001A48C0467944097949008F442201171AE9
:10010000E16803220A40032A00D01548E168490645
:10011000490F491C00F035FEE1684904490E484387
:10012000E168490F491C00F02CFE0AE07D20000226
:1001300007E00120C00304E020688004410F084864
:10014000C84008490860A26892093C231340064A47
:10015000D258D040086010BD0010024000127A0052
:0C0160000024F400000000206C010008E6
:10016C000000000000000000000000000000000083
:10017C000000000000000000000000000000000073
:10018C000100000002000000030000000400000059
:10019C000600000007000000080000000900000035
:1001AC00F0B591B00023102B03D0C45CD4545B1C6D
:1001BC00F9E7A2480160A24802600022A148102A77
:1001CC000BD08B5C835483188C1865785D70A57884
:1001DC009D70E478DC70121DF1E70421994C2C29F8
:1001EC0048D08D000C22102A06D0A35C10AEB61895
:1001FC000C3E3370521CF6E710AEF778B378727879
:10020C003678880703D00F970E93134612E08E486A
:10021C000D910146865D10A80F96C670CE5D0E96A8
:10022C008670CB5C43708A5C0D998E08874FBE5DDF
:10023C0056400670834F7A1910461038007870407B
:10024C0078550120284316460F3E36785E403E54C2
:10025C000220284313460E3B1B780E9E73403B54E2
:10026C00032028430D3A12780F9B5A403A54241D10
:10027C00491CB4E70A2000F0EDF80920744C0090FA
:10028C006F480068417B427A4273427943784371EC
:10029C00427241708178827A827081728179827B1C
:1002AC0082718173C178C279C270C27AC271C27B09
:1002BC00C173C272002104290AD00022102A04D072
:1002CC00835CE35C8354121DF8E7401C491CF2E785
:1002DC000099080600D1ADE0C8B200F0BBF8584850
:1002EC00006807900020102800D1A0E0079F3A5624
:1002FC00D109144604921B2211400B460F9060004A
:10030C00434059001E4605934BB2DB09134040B2E3
:10031C00C0091040484041000546069059400E91D6
:10032C000F98391801200F560B46022009561C460F
:10033C0003930846784070400323E3560C935840CF
:10034C00FB0913407C000D9463400A9358406840AD
:10035C00CB0913404D006B400B935C0001946DB2C4
:10036C00EE0916406640704002960E9B58400A9B60
:10037C005C0065B2EB0913400D9D6DB2ED091540A3
:10038C00654009956C005C4008946040019B5BB231
:10039C00DB09134074005C400D9460400C9BDC093D
:1003AC0014405B005C4065006EB2F60916405BB20F
:1003BC00DB0913406B405A00724050400F9D079E62
:1003CC0070550846049D68400C9E70400A9E704013
:1003DC000B9E7040099E70400E9E70405840089EC7
:1003EC0070400D9E70405040039E70700F986F408F
:1003FC006740174C0E9D6F407940059D6940099DE3
:10040C0069405940089D69400D9B59405140F1701D
:10041C000C994F400B994F4006994F4002994F4011
:10042C006F400D994F405740B770001D5BE7009827
:10043C00401E24E700F00EF811B0F0BD14000020AF
:10044C000C00002018000020D40E0008CE0D00086F
:04045C00D40F0008B1
:1004600030B500010A4908180A4909680022042A1F
:100470000CD00023042B05D0C45CCD5C6540CD546A
:100480005B1CF7E7091D001D521CF0E730BDC0469C
:08049000180000200C00002000
:10049800D0B502AFFFB089B06E4600F031FA012046
:1004A8000104B160F061C0077060E648006830611F
:1004B800E54800F033FB7F280FD080B2E34988423B
:1004C80003D0E349884200D1FFE1DE480068316982
:1004D800401ADD498842EBD9F7E100F032FCFC48CC
:1004E80000F01CFB0546401CF9D0A8B2D849884248
:1004F800DED0F74800F012FB0028F0D4FF2181433A
:10050800E8B2022813D1022911D1FC488019F169F7
:100518004170792101700171EE4A1178C1705178EA
:100528000F220A408270052100F08AFBD7E70246B5
:100538000A4321D1F14880197921817392224273AB
:10054800822202737322C27263228272432242722F
:10055800312202722122C271112282710223437157
:10056800F36903710023C37082700B22427001701B
:100578000F2100F065FBB2E7112813D1112911D121
:10058800FF2500F0DEFB0024D84804710460052C28
:1005980017D0CF4800F0C2FA0028A0D4D349085594
:1005A800641CF4E701282BD1012929D1D3488019EB
:1005B800792101710022C27082701122427001708B
:1005C800B1E7CA4CE078A1786278237853404B4071
:1005D8004340206800BA20602079834200D0C8E0F8
:1005E80000F0AFFB0024022C46D0B94800F096FA80
:1005F800002800D573E7C14989190855641CF2E73A
:10060800432823D1432921D100F09BFBB04800F0B7
:1006180085FA002800D562E70246093207218A4395
:100628006946F16069468A1A95467061851C1446C8
:10063800B261002D4AD0A64800F070FA002800D513
:10064800A3E02070641C6D1EB269F2E7312832D134
:10065800312930D100F075FB0024A44804710460EE
:10066800052C70D09A4800F059FA002800D536E7D2
:100678009E490855641CF3E7A048801944786C40EB
:100688000078A04275D1254608350720854300F03B
:1006980058FB6846B0616846451BAD46641CEC22B1
:1006A8002846214600F086FB2846214600F0C8FA75
:1006B800B069854613E700F04EFB8B480068316946
:1006C800401A8349884200D809E7FEE07169481C4E
:1006D800C9B20346804D002B04D014786140521CE7
:1006E8005B1EF8E7B269105C814245D1E8680028D2
:1006F80003D57A4828607B4828600020B46871696F
:1007080088423CDC115C06291BD3AA682242FCD132
:10071800AA68AA603F22D200EB689343EB60C90045
:10072800EA680A43EA60EA6802210A43EA60EA687A
:100738002243EA60AA682242FCD1EA688A43EA6056
:10074800B269401CDBE7694A1078517841409078DB
:100758004840D1784140107981420AD100F0F1FA3D
:100768005B4800F0DBF9002800D5B8E6411C8A0791
:100778000ED000F0F0FAB2E600F0EDFA05E0E86815
:1007880071680843E86000F0DCFAF0688546A6E680
:100798007061B161F069010258488019FF22F16067
:1007A80000F008FB00254E4CB069A84209D0484823
:1007B80000F0B4F9002804D45049891948556D1C33
:1007C800F2E72068C00701D0142000E00420F16996
:1007D80021507469A54200DC81E63D4800F09EF98D
:1007E800002800D57BE600212246A14205DC434BC8
:1007F8009B195B5C5A40491CF7E7D1B28142B8D1DA
:100808003A49086800BA08603949884200D264E663
:1008180000193849884200D95FE6F01D1930F1689F
:1008280000F0C7FA00242C4D7069844212DC33486A
:1008380080190019F11D19310A192F49FFF7B2FC67
:100848001034F1E71000002088130000FFFF0000BB
:10085800FEFF0000E868002803D5204828602148EA
:100868002860B069C010F0600021B468F068814267
:1008780022DAAA682242FCD1AA68AA60B161CA0039
:10088800F31D19339C18606870619B5817480568F8
:100898001148C068F4692043B4680F49C860AB5078
:1008A800A8180D46BFF36F8F71694160A868204290
:1008B800FCD1B169491CD9E7E868F1698843E86067
:1008C800E86871680843E86007E600F06DF9ECE550
:1008D80088130000005801400820024023016745A2
:1008E80014040050AB89EFCD100000200400002054
:1008F80000300008FFEF0108D410000820010000B4
:10090800F0B583B0744800687D21C90000F035FA5D
:10091800401E010E0DD17149714A5060714803683B
:100928000B400321890759180160002090600720B7
:1009380010606D4E37680020C04302906B496C4AC6
:10094800754C0D46BF35106828420AD13068C01B67
:10095800A042F6D33220029900F082F9644A634932
:10096800EFE7506B072101435163624A1068032384
:100978009843106010680C2101918843106010683A
:10098800012738431060106804210143116098065C
:1009980059490A6882430A60B8060A6802430A602D
:1009A800780388613E0455488169C9B2AA2903D0F1
:1009B8008169C9B2CC2929D1C168002903D5504918
:1009C800016050490160C168490003D54E49416042
:1009D8004E4941608169FF22914381618169EC221E
:1009E8000A43826181683142FCD11C467904C2689D
:1009F8000A43C26081683142FCD1F906C2680A43E1
:100A0800C2606420029900F02BF92346CF208104AC
:100A180034460526300702688A4302604521C90426
:100A280002680A4302601905C2688A43C260390530
:100A3800C2680A43C2600F210A02436A93434362B1
:100A48003A02436A13434362426AF0239A4342627A
:100A5800426A1023134343620904426A8A4342628A
:100A6800416A029421434162B903214A106C084348
:100A7800106427480268BA4302603A070368934340
:100A880003603A03036813430360FA03036893435C
:100A9800036002682A4302600268019B1A430260ED
:100AA80002681C4B1343036082680A4382600F4943
:100AB800C1600168394301600E4D002E0AD0AF6154
:100AC800962000F0EFF80298A861962000F0EAF866
:100AD800761EF2E703B0F0BD00000020FFFFFF0024
:100AE80010E000E020ED00E01000002041030000CD
:100AF8000010024000040050000800500820024086
:100B080023016745AB89EFCD3B2A19087F6E5D4C01
:0C0B1800003801400000FF0389130000BA
:100B2400F0B51E4A146813681D491F4D0E68B606B9
:100B340011D41668F61A86420DD21668361B4B2E4F
:100B4400F4D314682E68F60701D0142600E00426B6
:100B540001277751EAE71268D21A82420FD211486C
:100B64000A6812070FD40A6852070ED40A6892075B
:100B74000DD40A68D2070CD18868C0B20BE00020FB
:100B8400C043401E07E0082204E0042202E00222DF
:100B940000E001224A6000B2F0BDC046100000200F
:0C0BA4001C380140FFFF0000140400504A
:100BB000F0B581B0012002031A490B6813430B60A2
:100BC000194B9C6804439C6000241848184D1D4E26
:100BD000AC4205D227583FBA1F602418A419F7E782
:100BE000144C24681B68A34215D10B6893430B6017
:100BF000124900248C604C600C6072B61049086089
:100C0000016881F3088862B640688047E1437D202F
:100C100000F02AF8FAE7FA20074900F025F801B0B9
:100C2000F0BDC046381002400030024000300008DD
:100C3000FCBF0100FCEF01088813000010E000E099
:080C400008ED00E004D0FFF70D
:100C480010B50022054B8A4206DA1C682406FCD53A
:100C5800845CDC60521CF6E710BDC0461C380140BD
:100C6800F0B581B000910546012630040B4F38607D
:100C78000B4804680A480068001B009988420AD299
:100C880002203860284600F00DF8700438602846C5
:100C980000F008F8EEE701B0F0BDC04618040050B7
:040CA8001000002018
:100CAC0081B005490A6800920A68009BD21A8242F8
:0C0CBC00FAD301B07047C04610000020C1
:100CC80002480168491C01607047C04610000020B6
:100CD800034C206804348047FBE7FFF7D9FBFEE7A5
:040CE800E41000080C
:020CEC00FEE721
:020CEE00FEE71F
:020CF000FEE71D
:020CF200FEE71B
:020CF400FEE719
:020CF600FEE717
:020CF800FEE715
:020CFA00FEE713
:020CFC00FEE711
:020CFE00FEE70F
:020D0000FEE70C
:020D0200FEE70A
:020D0400FEE708
:020D0600FEE706
:020D0800FEE704
:020D0A00FEE702
:020D0C00FEE700
:020D0E00FEE7FE
:020D1000FEE7FC
:020D1200FEE7FA
:020D1400FEE7F8
:020D1600FEE7F6
:020D1800FEE7F4
:020D1A00FEE7F2
:020D1C00FEE7F0
:020D1E00FEE7EE
:020D2000FEE7EC
:020D2200FEE7EA
:020D2400FEE7E8
:020D2600FEE7E6
:020D2800FEE7E4
:020D2A00FEE7E2
:020D2C00FEE7E0
:020D2E00FEE7DE
:060D3000FFF7CEF9D0E749
:0E0D360080B50020C143FA20FFF793FF80BD77
:060D4400002000217047B1
:100D4A0000B581B06846792101700121FFF777FF6C
:040D5A0001B000BD27
:100D5E0000B581B068461F2101700121FFF76DFFBC
:040D6E0001B000BD13
:100D720080B57D2080000021C943FFF774FF80BD4C
:100D82000A0015D00300400800E052008242FCD95C
:100D9200002000E052089B1A06D340418A42F9D152
:100DA200704752089B18F8D200188A42F9D170474E
:080DB20010B5FFF7C6FF10BDEC
:100DBA0000220B0011001A00002A02D0013A8154C5
:040DCA00FCD17047A1
:100DCE008D01020408102040801B366CD8AB4D9A62
:100DDE002F5EBC63C697356AD4B37DFAEFC59139E1
:100DEE0072E4D3BD61C29F254A943366CC831D3A0B
:100DFE0074E8CB8D01020408102040801B366CD89D
:100E0E00AB4D9A2F5EBC63C697356AD4B37DFAEFAD
:100E1E00C5913972E4D3BD61C29F254A943366CC25
:100E2E00831D3A74E8CB8D01020408102040801B0C
:100E3E00366CD8AB4D9A2F5EBC63C697356AD4B369
:100E4E007DFAEFC5913972E4D3BD61C29F254A94F4
:100E5E003366CC831D3A74E8CB8D01020408102052
:100E6E0040801B366CD8AB4D9A2F5EBC63C697354F
:100E7E006AD4B37DFAEFC5913972E4D3BD61C29FD6
:100E8E00254A943366CC831D3A74E8CB8D01020457
:100E9E0008102040801B366CD8AB4D9A2F5EBC6379
:100EAE00C697356AD4B37DFAEFC5913972E4D3BDD6
:0F0EBE0061C29F254A943366CC831D3A74E8CBFA
:040ED000E100000835
:100ED400637C777BF26B6FC53001672BFED7AB76F3
:100EE400CA82C97DFA5947F0ADD4A2AF9CA472C09E
:100EF400B7FD9326363FF7CC34A5E5F171D831150B
:100F040004C723C31896059A071280E2EB27B2752B
:100F140009832C1A1B6E5AA0523BD6B329E32F84A3
:100F240053D100ED20FCB15B6ACBBE394A4C58CF9B
:100F3400D0EFAAFB434D338545F9027F503C9FA86F
:100F440051A3408F929D38F5BCB6DA2110FFF3D23D
:100F5400CD0C13EC5F974417C4A77E3D645D1973F1
:100F640060814FDC222A908846EEB814DE5E0BDBEB
:100F7400E0323A0A4906245CC2D3AC629195E47922
:100F8400E7C8376D8DD54EA96C56F4EA657AAE087C
:100F9400BA78252E1CA6B4C6E8DD741F4BBD8B8A17
:100FA400703EB5664803F60E613557B986C11D9E7D
:100FB400E1F8981169D98E949B1E87E9CE5528DFF4
:100FC4008CA1890DBFE6426841992D0FB054BB1620
:100FD40052096AD53036A538BF40A39E81F3D7FBAA
:100FE4007CE339829B2FFF87348E4344C4DEE9CBF4
:100FF400547B9432A6C2233DEE4C950B42FAC34E69
:10100400082EA16628D924B2765BA2496D8BD1251E
:1010140072F8F66486689816D4A45CCC5D65B692C2
:101024006C704850FDEDB9DA5E154657A78D9D8466
:1010340090D8AB008CBCD30AF7E45805B8B3450686
:10104400D02C1E8FCA3F0F02C1AFBD0301138A6BA0
:101054003A9111414F67DCEA97F2CFCEF0B4E673D0
:1010640096AC7422E7AD3585E2F937E81C75DF6E7E
:1010740047F11A711D29C5896FB7620EAA18BE1BE4
:10108400FC563E4BC6D279209ADBC0FE78CD5AF48A
:101094001FDDA8338807C731B11210592780EC5FD0
:1010A40060517FA919B54A0D2DE57A9F93C99CEF2C
:1010B400A0E03B4DAE2AF5B0C8EBBB3C835399612D
:1010C400172B047EBA77D626E169146355210C7D6B
:1010D400046062063E0B5C4E040620504F34414BC4
:1010E4001511000804000020050000001511000877
:1010F4000C000020BC0000002711000800000020A4
:0C1104001011000804000000E30C0008BB
:041110000024F400C3
:10111400206861680834002200E042540139FCD59B
:02112400704712
:1011260020686168A2680C3401E08B5C8354013A44
:04113600FBD570472E
:0400000508000D31B1
:00000001FF
